:100000000428FF3FFF3FFF3F0130031383129F008F
:100010000E3083169F00013085008601870188011C
:1000200089018312850186018701880189012008E1
:100030008600013088001F150230FB00FF30FA00F7
:10004000FB0B23282628FA0B232820284A30FA0005
:10005000FA0B282883161E088312A8070208A8078F
:1000600021088600023088001F150230FB00FF3097
:10007000FA00FB0B3C283F28FA0B3C2839284A3071
:10008000FA00FA0B412883161E088312A9070208FA
:10009000A90722088600043088001F150230FB00E3
:1000A000FF30FA00FB0B55285828FA0B5528522828
:1000B0004A30FA00FA0B5A2883161E088312AA0740
:1000C0000208AA0723088600083088001F1502309E
:1000D000FB00FF30FA00FB0B6E287128FA0B6E282C
:1000E0006B284A30FA00FA0B732883161E08831215
:1000F000AB070208AB0724088600103088001F15E4
:100100000230FB00FF30FA00FB0B87288A28FA0B2D
:10011000872884284A30FA00FA0B8C2883161E0898
:100120008312AC070208AC0725088600203088003F
:100130001F150230FB00FF30FA00FB0BA028A3289C
:10014000FA0BA0289D284A30FA00FA0BA52883163E
:100150001E088312AD070208AD072608860040304E
:1001600088001F150230FB00FF30FA00FB0BB92896
:10017000BC28FA0BB928B6284A30FA00FA0BBE2878
:1001800083161E088312AE070208AE0727088600F2
:10019000803088001F150230FB00FF30FA00FB0B97
:1001A000D228D528FA0BD228CF284A30FA00FA0BE9
:1001B000D72883161E088312AF070208AF07B00ABC
:1001C00030081F3A031D6529A00D2010A10D211034
:1001D000A20D2210A30D2310A40D2410A50D25108F
:1001E000A60D2610A70D27100730F4002808F000F0
:1001F00067217808F0007008B1007008003A031D0C
:10020000022920140730F4002908F000672178083B
:10021000F0007008B1007008003A031D1029211485
:100220000730F4002A08F00067217808F000700811
:10023000B1007008003A031D1E2922140730F40093
:100240002B08F00067217808F0007008B1007008F2
:10025000003A031D2C2923140730F4002C08F00069
:1002600067217808F0007008B1007008003A031D9B
:100270003A2924140730F4002D08F000672178088B
:10028000F0007008B1007008003A031D48292514D9
:100290000730F4002E08F00067217808F00070089D
:1002A000B1007008003A031D562926140730F400E7
:1002B0002F08F00067217808F0007008B10070087E
:1002C000003A031D64292714B00117286629031377
:1002D0008312F8010830FC00700DF80D7408F80264
:1002E00003187429F8070310F00DFC0B6C290800A3
:02400E003A3F37
:00000001FF
